:020000040000FA
:10000000C0230020150200001D0200001F02000096
:100010002102000023020000250200000000000071
:1000200000000000000000000000000027020000A7
:1000300029020000000000002B0200002D02000039
:100040002F0200001D0300002F0200002F020000FD
:100050002F0200002F0200002F0200002F020000DC
:100060002F0200002F0200002F0200002F020000CC
:100070002F0200002F0200002F0200002F020000BC
:100080002F0200002F0200002F0200002F020000AC
:10009000790300002F0200002F0200002F02000051
:1000A0002F0200002F020000ED0600002F020000CA
:1000B0002F0200002F0200000000000000000000DE
:1000C0002F0200002F0200002F0200002F0200006C
:1000D0002F0200002F0200002F020000000000008D
:1000E0000000000000000000000000000000000010
:1000F0000000000000000000000000000000000000
:1001000000000000000000000000000000000000EF
:1001100000000000000000000000000000000000DF
:1001200000000000000000000000000000000000CF
:1001300000000000000000000000000000000000BF
:1001400000000000000000000000000000000000AF
:10015000000000000000000000000000000000009F
:10016000000000000000000000000000000000008F
:10017000000000000000000000000000000000007F
:10018000000000000000000000000000000000006F
:10019000000000000000000000000000000000005F
:1001A000000000000000000000000000000000004F
:1001B000000000000000000000000000000000003F
:1001C000000000000000000000000000000000002F
:1001D000000000000000000000000000000000001F
:1001E000000000000000000000000000000000000F
:1001F00000000000000000000000000000000000FF
:10020000DFF80CD000F03CF8004800476D09000012
:10021000C02300200648804706480047FEE7FEE767
:10022000FEE7FEE7FEE7FEE7FEE7FEE7FEE7FEE7A6
:10023000D10300000102000040EA01039B0703D044
:1002400009E008C9121F08C0042AFAD203E011F815
:10025000013B00F8013B521EF9D27047D2B201E0D7
:1002600000F8012B491EFBD270470022F6E710B5BB
:1002700013460A4604461946FFF7F0FF204610BD14
:10028000064C074D06E0E06840F0010394E80700E3
:1002900098471034AC42F6D3FFF7B6FFA81700001A
:1002A000C817000000F01F020121914040098000A2
:1002B00000F1E020C0F88012704700F01F02012119
:1002C00091404009800000F1E020C0F880117047A3
:1002D00000F01F02012191404009800000F1E02060
:1002E000C0F80011704700F01F0201219140400941
:1002F000800000F1E020C0F8001270474907090EA5
:10030000002806DA00F00F0000F1E02080F8141D4C
:10031000704700F1E02080F80014704770B5144C6D
:10032000D4F80001002628B1D4F80403C00701D096
:10033000C4F80061D4F80C010E4D40B1D4F80403A8
:10034000000704D5C4F80C61286900B18047D4F8CF
:10035000100100280BD0D4F80403C00607D5C4F858
:100360001061E868002802D0BDE87040004770BD09
:1003700000100040040000207CB5144C606A01901D
:100380002078002821D00120FFF797FF656800261C
:1003900066600120FFF79CFFE169002915D0E8079E
:1003A00003D08DF8006068468847A80705D501206E
:1003B0008DF80000E16968468847680705D5022086
:1003C0008DF80000E169684688477CBD0400002084
:1003D000F0B5B5480023021D0178101D01254FF02E
:1003E000805406290BD11678360708D10678C6F353
:1003F0000316032E06D0042E04D0052E02D00629A3
:1004000007D00EE0B4F82463A84FC6F304263E607C
:1004100002E01678360704D10678C6F30316032ED9
:1004200002D0062904D00FE0A24FA14E7E670EE055
:100430001678360708D10678C6F30316032E06D0C1
:10044000042E04D0052E02D0062907D00EE0D4F8E1
:100450004462994FC6F342363E6002E01678360792
:1004600004D10678C6F30316032E02D0062906D05F
:1004700011E0924E376827F0807737600EE01678EB
:10048000360708D10678C6F30316032E06D0042ECD
:1004900004D0052E02D006290AD011E04FF0804684
:1004A000C6F80C31C6F81031834E361F336002E0B7
:1004B0001678360704D10678C6F30316032E02D049
:1004C000062905D00CE07C4F032664373E600AE025
:1004D0001678360704D10678C6F30316032E02D029
:1004E00006290DD014E0764F05263E60744E78360E
:1004F0003560734E083633603F263F1D3E6002E094
:100500001678360704D10678C6F30316052E02D0F6
:10051000062957D062E06B4E36686B4F3E60694EDD
:10052000361D36683F1D3E60664E083636683F1DF4
:100530003E60644E0C3636683F1D3E60614E10369C
:1005400036683F1D3E605F4E143636683F1D3E6084
:100550005C4E183636685C4F20373E60594E1C366C
:1005600036683F1D3E60574E203636683F1D3E6060
:10057000544E243636683F1D3E60524E283636684B
:100580003F1D3E604F4E2C3636683F1D3E604D4E3F
:10059000303636684C4F40373E604A4E3436366807
:1005A0003F1D3E60474E383636683F1D3E60454E23
:1005B0003C3636683F1D3E60424E403636683F1D31
:1005C0003E6002E01678360708D10678C6F30316B7
:1005D000032E06D0042E04D0052E02D0062907D003
:1005E00019E0D4F85812394A01F04F01116002E0C5
:1005F000117809070FD10078C0F30310032803D046
:10060000042801D0052806D131480168C90702D065
:100610006FF001010160D4F83001062808D1D4F848
:100620003401062804D12B48016841F4806101603F
:1006300022487438016841F470010160BFF34F8FA4
:10064000BFF36F8F4FF01021D1F80002002803DBB9
:10065000D1F80402002822DA1F4A15601F480468F6
:10066000002CFCD01524C1F800420568002DFCD0F8
:10067000C1F8044201680029FCD013600168002918
:10068000FCD0BFF34F8F0D48F0380168144A01F4D5
:10069000E06111430160BFF34F8F00BFFDE71249D6
:1006A00010480860F0BD0000E00F00F04035014048
:1006B0000DF0ADBA00C007403C050040FCED00E085
:1006C000105600400404001020C50040E40E004015
:1006D000000400403C17004004E5014000E40140F4
:1006E0000400FA050090D0034C0000200748D0F821
:1006F0004011002909D00021C0F840110448407879
:10070000032802D1034901200861704700A001407D
:10071000040000200010004002E008C8121F08C1B9
:10072000002AFAD170477047002001E001C1121F72
:10073000002AFBD17047006890FAA0F000BA00BA16
:100740007047000072B609480068C00700D000BEBC
:10075000BFF34F8F0548E4380168054A01F4E061B2
:1007600011430160BFF34F8F00BFFDE7F0ED00E0E4
:100770000400FA050EB500210091CDE901106A468A
:1007800044F20100FFF7DEFF0EBD000006480168DD
:1007900021F0010101600548016821F0010141F0EB
:1007A00080710160002070475016004074170040AF
:1007B0002DE9FC410646C0074FF000050ED0104F52
:1007C00000240122385D009500231146019500F0B8
:1007D0001FFC641C042CF4D300F01CF8B0070DD5EA
:1007E000074E0024361D0022305D0323009511467C
:1007F000019500F00DFC641C042CF4D3BDE8FC81D1
:10080000A01700000249085C012100F01EBC000096
:10081000A017000010B500242046FFF7F3FF641C6A
:10082000042CF9D310BD006890FAA0F000BA70470C
:1008300070B50F4D0F4CA868C4F800020E486969E6
:10084000C07C88470E490D4808600021C4F810118B
:1008500001202061D4F81021002AFBD0C4F8101127
:10086000A96841F00401C4F80012606070BD000086
:1008700004000020001000409C0000207E030020A7
:10088000041500404FF080400021C0F80011012104
:10089000C0F80010D0F800110029FBD0704700000C
:1008A00010B51CA08AB0006808901BA01BA10068AE
:1008B0000990D1E90001CDE90601182219496846DD
:1008C000FFF7BAFC00208DF8140003208DF8130008
:1008D0000124154801908DF808408DF801406846C4
:1008E00000F00EF9002812D108A800F043FA002801
:1008F0000DD109A800F06CFA002808D1082106A83B
:1009000000F0ACFA002802D10848047000200AB0B8
:1009100010BD0000E7E7E7E7C2C2C2C2E7C2C3C436
:10092000C5C6C7C888170000010A00005000002093
:1009300010B50D4C012020706070A070E070FFF7C2
:1009400037FF2178112000F075FB6178122000F04C
:1009500071FBA178132000F06DFBE178BDE8104039
:10096000142000F067BB000000000020FFF7E0FF4C
:10097000FFF796FF08B1FFF7FDFEFFF783FF00F0DA
:10098000B1FA08B1FFF7F6FE0A480178427841EA69
:1009900042018278C078920042EAC00001430648D2
:1009A000417100F0DFFA08B1FFF7E4FE20BF40BF5D
:1009B00020BFFBE7000000205000002070B50C496C
:1009C0004FF4705008600B4C0025657000F01EFD60
:1009D00020210948FFF749FCE56214202563FFF751
:1009E0006CFC06490320C1F80002002070BD000025
:1009F00008F5014004000020A00300200010004082
:100A000010B5007800285ED0012814D002285AD1F1
:100A10002D4800F06BF90028FAD02B482B4C407978
:100A200000F00F0001280AD0022810D004283AD084
:100A3000082813D13FE0BDE8104000F049B8207805
:100A400018B100212170112006E00121FAE7607839
:100A500038B300216170122000F0ECFA21781120E7
:100A600000F0E8FA6178122000F0E4FAA17813208F
:100A700000F0E0FAE178142000F0DCFA12480121DD
:100A80002538017021786278E37841EA4201A27842
:100A9000920042EAC30211434171BDE8104000F0E8
:100AA00061BA0121D6E7A07818B10021A170132006
:100AB000D2E70121FAE7E07818B10021E1701420B3
:100AC000CAE70121FAE710BD7500002000000020F0
:100AD000094810B5007860B10120FFF7EEFB074828
:100AE00000218162016241620120FFF7F1FB0020D9
:100AF00010BD082010BD000004000020DC01002013
:100B00002DE9F04105007DD0694C207818B1FFF740
:100B100055FF002877D16868E061182229466548AA
:100B2000FFF78AFB0025656020216348FFF79DFBE6
:100B3000E562256300F0AEFD00287DD05F494FF0EF
:100B4000E7300860091D4FF043300860091D5C481C
:100B50000860091D5B48086000F058FC55490020FA
:100B6000183101F5947200BF00EB800303EB4013D2
:100B70000B4442F82030401C0828F5DB5249002085
:100B800001F5947200EB800303EB40130B4442F831
:100B90002030401C0828F5DB4C48042606604B48F2
:100BA000083805604A4840F20221C0F800124A4A5B
:100BB00048491160111D0860DFF81881091D08F10E
:100BC0000408C1F80080001D091D0860091D434884
:100BD00008604048F038091D08604048001D091DA4
:100BE0000860091D3E480860324F787C00F007011C
:100BF0000120FFF783FBB87C00F007011420FFF70A
:100C00007DFB01E04FE04CE01420FFF761FBA07892
:100C10000127E8B3A068294940F04000A060022005
:100C2000443108602F49032008602E4808300660D0
:100C30002C490520383100E037E008602A4E40F2A8
:100C40000110C6F800022748001F05603804C6F8E6
:100C50000403F76005211A20FFF750FB1A20FFF765
:100C600037FB1D490839C1F80080081D0660194886
:100C70001949283010390860174A311D0C3A1160A3
:100C800015491839086018480C30091D086000E043
:100C900004E011494FF460705C390860657027709A
:100CA0000020BDE8F0810E20FBE70720F9E70000F7
:100CB000040000209C000020A00300201C15004020
:100CC000E743C323A363E3130802002010A50040F9
:100CD00000A000400011004060F5014040A100402C
:100CE0000010004008A5014000A0014070B5054675
:100CF0001E48007880B385B31D4CA06A70B30120F4
:100D0000FFF7DBFA606A54F820100A782A7054F86A
:100D100020104978697054F820108978A97054F827
:100D200020100979297154F82010C978E97054F815
:100D30002010681D491DFFF77FFA606A401C606241
:100D4000082801D300206062A06A401EA062012032
:100D5000FFF7BEFA002070BD01E002E003E00820CA
:100D6000F9E70E20F7E70520F5E700000400002072
:100D70003003002070B5134E0446707808B111207E
:100D800070BDCCB10F483430407C052816D04FF0F0
:100D90007F452046FFF7CFFC284204D10A4800686F
:100DA00010F0FF0F0CD020687063012000F02EFCC3
:100DB000BDE87040FFF7EABC0E2070BD034DE8E7C8
:100DC000072070BD04000020241500400000FFFF34
:100DD00070B51F4D0446687808B1112070BD84B30A
:100DE0001B483430407C05282DD04FF07F462046EC
:100DF000FFF7A1FC30421BD11649086810F47F4F61
:100E000023D0086810F47F0F1FD00868000E1CD094
:100E1000091D0868000E18D0086810F47F0F14D060
:100E2000086810F47F4F10D0086810F0FF0F0CD046
:100E30002068A863022000F0E9FBBDE87040FFF7DE
:100E4000A5BC0E2070BD044ED1E7072070BD000088
:100E500004000020241500400000FFFF70B50C4680
:100E60001D49497809B1112070BDB0B1092C31D2AA
:100E7000194D3435697C052911D04FF07F412CB1D3
:100E8000164A12680A4201D102781AB3134A121D97
:100E900012680A420BD1012107E00E2070BD1049F3
:100EA000EDE7425CB2B1491CC9B2A142F9D3014697
:100EB000094822463C30FFF7BFF9C4F10801FF2082
:100EC0002C74C840A874042000F0A0FBBDE870405A
:100ED000FFF75CBC072070BD040000201C1500401B
:100EE0000000FFFF70B51A48417809B1112070BDAC
:100EF000184C4FF0FF31C4F808130025C4F8105106
:100F00001549C160816841F00401C4F80012102144
:100F1000C4F80413042141700D48104A3430817C18
:100F200011600E49C07C28390860091F0C48086010
:100F300001209434FFF7B6F90120FFF7C9F92567BE
:100F40006567E567012044F8900C002070BD000043
:100F50000400002000100040611000003015004027
:100F60007E0300202DE9F041264F0546387840B138
:100F700055B1287868B120280BD8234E317829B193
:100F800009E00820BDE8F0810E20FBE7F17C8842F3
:100F900001D90920F6E71D4CA06A082801D30420D6
:100FA000F0E76878082801D30720EBE70120FFF776
:100FB00084F9206A2522294654F82000FFF73CF9DD
:100FC00010486A782C30815C491C01F0030181547F
:100FD000206A54F82020401C08281171206201D397
:100FE00000202062A06A401CA0620120FFF770F977
:100FF000707828B9307C18B9787808B900F060FAB0
:101000000020BFE7040000209C000020DC0100203D
:1010100070B541EA4201DDE904564FF0A04441EACF
:10102000830141EA052104EB800041EA0641C0F852
:10103000001770BD01224FF0A043824011B1C3F8E8
:1010400008257047C3F80C25704701224FF0A043D4
:10105000824011B1C3F808257047C3F80C257047CA
:101060002DE9F05F554800220127006818B1544867
:10107000806A082803D3BDE8F05FFFF7D9BBDFF82B
:101080003C9109F10809D9F800004D49703101EB94
:10109000800609F104010C68494B35884E33AC4297
:1010A000587805D1B478B4EB500F01D10122002754
:1010B0004008B07008689A4630804248424C017D32
:1010C00019B19AF80110C90710D0A1683F4B41F03F
:1010D0000801C3F800123C49394D007849694FF0C6
:1010E000000B2C35B8B3012847D102E0FFF7A0FB75
:1010F0004EE03748836AB3F1000E2DD0436A50F8B2
:1011000023C09CF80180D9F800C0E04524D196F8AE
:1011100003C0BCF1010F0DD162B95B1C4362082B07
:1011200001D3C0F824B0AEF101028262626842F0DD
:10113000010262600122F270426A50F82200A0614E
:1011400000788847A1690878287011F8052BA81C39
:10115000FFF772F806E009E086F803B00020884740
:1011600085F800B09AF80100687006E00020884712
:101170009AF80000287085F801B005206070D9F851
:101180000000144908601348283805601248E060E0
:10119000002F10D0B178D9F80000C0B200F044F9A7
:1011A000002808D0606840F004006060BDE8F05F8F
:1011B0001420FFF798B8BDE8F09F0000001400402D
:1011C000300300209C00002004000020001000409C
:1011D000DC0100202C150040DD11000010B5094C89
:1011E0000949A06840F00400C1F80002074861699D
:1011F000C07C88470749064808600748E06004202B
:10120000607010BD04000020001000409C00002011
:101210007E030020041500406110000070B5164CDC
:10122000164AA068C2F80002A06A15490860154B6A
:10123000091D9889823808601348012140F80C1F65
:101240000021C0F83411C0F83811104D4FF4E050AF
:10125000286050142D1D2860C2F80C11187810B9A0
:101260006169002088470B49094808600A48E06026
:101270000320607070BD00000400002000100040DA
:1012800040A500409C00002000A0004004F5014063
:101290007E03002004150040D912000010B50C4C4C
:1012A000606840F00100606000F096F90948806ACB
:1012B00030B11420FFF717F8BDE8104000F000B976
:1012C00000206070BDE810401420FFF70CB800004B
:1012D00004000020DC0100202DE9F047414A4FF4D2
:1012E000E05010604049D1F80C31DFF80091002740
:1012F0003F4CB9F80E004E14DFF8F8800125E3B337
:101300003D4B1B68CBB365601660D8F8041041F004
:101310000101C8F80410D8F82010401A401CC8F881
:10132000240000F059F999F8000088B109F2E22090
:10133000017869B14078410830480068C0B200F0D7
:1013400073F828B1D8F8040040F00400C8F804008D
:101350002B48806A50B199F81000012806D014205B
:10136000FEF7C1FFBDE8F04700F0AAB888F80170A9
:10137000BDE8F0471420FEF7B6BFD8F820C0BCF196
:10138000010CC8F820C00BD265601660401CC8F87C
:101390002400D8F8040040F00200C8F80400E5E793
:1013A000D8F808000F4640F00802C1F80022D8F82B
:1013B0001800D8F8141000788847104811492838C8
:1013C00001601148C8F80C00022088F8010025606F
:1013D0000448001F0660D4F84401002800D03D6096
:1013E000BDE8F08708F50140001000409C00002097
:1013F00000A0004004000020001400402C15004014
:10140000DC0100205C0300201D12000005490020C3
:1014100008624862886201F5AA71086248628862BF
:1014200070470000DC0100202DE9F041224C074606
:101430008846A06A08283DD2A4F5257120460A787E
:101440000026006A01F2E225012A03D04A7842B15F
:10145000C97C02E0297820292CD854F8202011706A
:1014600002E054F820100E7054F82000A91C10F867
:10147000052BFEF7E1FE206A54F820104F700F494B
:10148000096854F82020917054F8202082F80480D4
:10149000697854F8202041F30001491C401CD170A8
:1014A0002062082800D32662A06A401CA0620120A6
:1014B000BDE8F0810020FBE7300300204815004024
:1014C0002DE9F05F3E4C4FF00108C4F824803D4800
:1014D000DFF8F4A0A0F5A077416A3C4D4FF0000B77
:1014E00050F82110A161387807F5307610B1012845
:1014F00044D10DE0087861698847A16908793070A6
:1015000086F801B011F8052BB01CFEF795FE18E027
:10151000C87828B3387D18B3002081460878307029
:1015200008794006000E7070CA78DAB100221043C4
:10153000707011F8052BB01CFEF77EFEB9F1000F9C
:1015400012D0A06840F00800C5F800021120C5F8CC
:101550000403F88920620220C4F80CA060700DE03A
:101560000120DAE70122E2E7A068C5F800021020B6
:10157000C5F804031648E06084F80180A069154AA4
:10158000417811604078444608FA00F0111D086067
:101590000B48104934302439C07C0860081F0660AD
:1015A0000120FEF77FFE0120FEF792FEC5F804B190
:1015B000C5F808B1C5F810B12C60BDE8F09F000077
:1015C00004000020DC0100201D120000001000407B
:1015D0009D1200002C15004010B50B4CA06A00288D
:1015E00011D00120FEF769FEA06A401EA062606A69
:1015F000401C6062082801D300206062BDE81040F2
:101600000120FEF765BE10BDDC01002010B50446C8
:10161000C00704D00F48FFF78EF80F490860A007F5
:1016200006D50C48001DFFF786F80B49091D086018
:1016300060070DD507480830FFF7F5F8064908316F
:10164000086004480C30FFF7EEF803490C310860DD
:1016500010BD0000380000201C1500400A48017A27
:101660000A4801600A4849B1012905D0032909D077
:10167000042901D000207047302100E04021816220
:10168000012070474921FAE79C0000201015004016
:101690000400002070B500F041F8FFF7DFFF194C9F
:1016A000194922787AB1012A0BD000220240607ACF
:1016B000B8B1164B1D1F01280ED0022807D00025F7
:1016C00013E0134A00E0134A4A610122EEE74FF6A5
:1016D000FF761E60104B03E0FF261E6040F20713EA
:1016E0002B600A4B083B1860012549691540E07CD6
:1016F0008847A089872801D3012000E000202840E6
:1017000070BD00009C000020040000203C1500403B
:101710005D17000031170000211001000248034945
:10172000807A0860704700009C0000200C15004083
:10173000084A074911600849497C491E090441EAE1
:101740000021014341F08070111D086070470000C6
:101750000001010014150040380000200749064828
:10176000086007480749407C401E41EA00400349A1
:10177000091D0860704700000600030014150040B2
:1017800038000020200000010100000000000000DF
:1017900001020000FA000300000102200000000026
:1017A000111213140D0E0F10C817000000000020B6
:1017B000500000001807000018180000500000201A
:1017C0007023000028070000000000000000010056
:1017D00000000000130100000000000000000000F5
:1017E00000000000000000000000000000000000F9
:1017F00000000000000000000000000000000000E9
:10180000E7E7E7E7C2C2C2C2E7C2C3C4C5C6C7C8EA
:081810000805FF020090D0035F
:0400000500000201F4
:00000001FF
